:1000000000308A0049290000FF00030E8301A1008F
:100010000A08A0008A010408A2007708A300780853
:10002000A4007908A5007A08A6007B08A70083131E
:1000300083128C308400801E1F288C1A32282208DC
:1000400084002308F7002408F8002508F900260892
:10005000FA002708FB0020088A00210E8300FF0E0B
:100060007F0E09008A110A12F6280A108A100A1156
:1000700082075B345B345C345B3445345D3441343B
:100080005B345C345B345B345E345F345F345D34EA
:1000900060345E345F345F3461340A108A100A11B0
:1000A00082070134F634F634F63401340034763401
:1000B00076347634893481347E347E347E34BD3473
:1000C00000347E347E347E348134003476347634A9
:1000D0007E347E340034F634F634FE34FE3481341B
:1000E0007E347634763485340034F734F734F7349C
:1000F00000347E347E3400347E347E34BE347E342C
:100100007E347E3480340034F734F734EB341C34DE
:1001100000347F347F347F347F340034FE34F03455
:10012000FE3400340034EF34DF34BF340034813423
:100130007E347E347E3481340034F634F634F63442
:10014000F93481347E347E347E3401340034F63424
:10015000F634F6340934B9347634763476348D3462
:10016000FE34FE340034FE34FE3480347F347F3479
:100170007F348034C034BF347F34BF34C0348034E3
:100180007F3480347F3480341C34EB34F734EB34E8
:100190001C34F834F7340734F734F8341E346E3432
:1001A00076347A347C34FF34FF34FF34FF34FF3448
:1001B000173433345534E634F734F034F734F73445
:1001C0000134F7343D345E346E347634793400349F
:1001D0007E347E347E340034F734F734F734F73429
:1001E000F73489347634763476348934831686014C
:1001F000553083128600BF013F08093C031C0929C2
:1002000028303F0784008C1E03291A088000BF0A8B
:10021000FC288C128A110A121F2839308400000829
:10022000031923290130F800BF30F7006400F70BF1
:100230001629F80B14294A30F700F70B1D29000086
:100240006400800B12290034F701F8013D08031007
:100250003E18F707F70CF80CBE18F707F70CF80C68
:100260003E19F707F70CF80CBE19F707F70CF80C56
:100270003E1AF707F70CF80CBE1AF707F70CF80C44
:100280003E1BF707F70CF80CBE1BF707F70CF80C32
:10029000003484011F3083056730831699002230B3
:1002A000980090308312980083161F149F141F1516
:1002B0009F1107309C00FF308312B40083161F107B
:1002C0009F141F159F151F1383121F179F17831647
:1002D0009F1383121F148316091283129412B412EF
:1002E0003408831687008312341634088316870077
:1002F0008312B411340883168700013083129400EE
:100300000030831694000108C739083881000F3087
:10031000F700073083128101813084000008F03932
:100320000738800064000008F739F719F0397704BE
:10033000800090010030F800920000308316920097
:1003400007309C00050864000230F700F70BA6296F
:10035000000000001C0883120D1383169D018C16EB
:10036000C03083128B040030F8001F08C7397804AE
:100370009F0083168601FF3083128600B301A80117
:10038000A8080319FE291F151F19C4291E08083CB7
:100390000318C3290A30B9000D21B6013608093CFB
:1003A000031CFD29B7013708043C031CF129283040
:1003B0003607840041300002BB00BD000530BE009E
:1003C0002421370878074D20B9008316860183124F
:1003D000390886006400A630F700F70BED29B70A4C
:1003E000D32983168601FF30831286006400A6306D
:1003F000F700F70BF929B60ACE29C029B50135084F
:10040000013C031C512AB8013808143C031C4F2A34
:100410001F151F19092A1E08083C0318082A0A304C
:10042000B9000D21B6013608093C031C462AB70164
:100430003708043C031C3A2A3508BD000A30BE00C8
:100440002421360878073520BF3EBC00BD000530AA
:10045000BE002421370878074D20B9008316860195
:100460008312390886006400A630F700F70B362A9D
:10047000B70A182A83168601FF30831286006400AB
:10048000A630F700F70B422AB60A132A3308B30A3C
:10049000783C03184D2A8A010028B80A042AB50AB4
:0604A000FF29C0296300E2
:02400E003D3F34
:00000001FF
